:100000000202AB75140AE4F515F51685172085185C
:1000100021758911F588F58AF58C7524F8F525F593
:10002000B0859031E59030E6036331FFE53130E78C
:10003000180514D3E514648094944003751414E5F2
:1000400014B40E1E75141980191514C3E5146480B8
:10005000948A500375140AE514B41006751407E465
:10006000F5B0E58CC394F84005E4F5888018E58C7C
:10007000D395244002800CE58CB5240AE58AD395FB
:1000800025400343B001E51464197095F588858A0D
:100090002CAF8CF5198F1AF58AF58C75881043B042
:1000A00003E51A751A00F519E52C251AF51AE43539
:1000B00019F519E590F4F51F531F30E51F700C7505
:1000C000260D752705752817752925E51FB4100C11
:1000D00075260E7527A675281A75290AE51FB420FE
:1000E0000C7526107527BE75281D7529C3E51FB42C
:1000F000300C7526137527887528227529B8E4F504
:100100000DF50CF50BF50AFCFDE50D251AF50DE5D1
:100110000C3519F50CED350BF50BEC350AF50AAE7F
:1001200020AF21AB07AA06C3E50D9BF50DE50C9AA0
:10013000F50CE50B9400F50BE50A9400F50A85191A
:1001400020851A21851910851A11E511AE10780540
:10015000CEC313CE13D8F9F5118E10251AF511E57B
:10016000193510F510D3E51A9527E519952650088D
:10017000E4F52DF52E020223C3E51A9529E519951C
:10018000285025851912851A13C3E5139527F513F1
:10019000E5129526F512E513AE127802CEA2E7130A
:1001A000CE13D8F8F5138E12AF90EFF4F52EE4F4D9
:1001B000F52D532E0F752D00E52EAE2D7807C33388
:1001C000CE33CED8F9F52E8E2D851908851A09E57E
:1001D00009AE087803CEC313CE13D8F9F5098E08FB
:1001E00085190E851A0FE50FAE0E7806CEC313CE15
:1001F00013D8F9F50F8E0E2509F523E508350EF510
:1002000022D3E52E9523E52D9522400685222D85C6
:10021000232ED3E52E9513E52D9512400685122D3C
:1002200085132EE485111E85101DF51CF51BFFFEA0
:10023000FDFCAB0DAA0CA90BA80AD312033740187A
:10024000E51E250DF51EE51D350CF51DE51C350BD0
:10025000F51CE51B350AF51BAE2DAF2EAB07AA0624
:10026000C3E51E9BF51EE51D9AF51DE51C9400F5E2
:100270001CE51B9400F51BAE17AF18E4FCFDAB1E8C
:10028000AA1DA91CA81BD312034D4008851715856C
:1002900018168006851D15851E1685152F851630A6
:1002A000E530F525E52FF524020021787FE4F6D826
:1002B000FD7581310202F2020003E493A3F8E49396
:1002C000A34003F68001F208DFF48029E493A3F849
:1002D0005407240CC8C333C4540F4420C8834004BB
:1002E000F456800146F6DFE4800B0102040810207A
:1002F000408090035EE47E019360BCA3FF543F30D6
:10030000E509541FFEE493A360010ECF54C025E01D
:1003100060A840B8E493A3FAE493A3F8E493A3C8D5
:10032000C582C8CAC583CAF0A3C8C582C8CAC58366
:10033000CADFE9DEE780BEEB9FF5F0EA9E42F0E916
:100340009D42F0EC6480C864809845F022EB9FF5F4
:10035000F0EA9E42F0E99D42F0E89C45F022021747
:03036000F80000A2
:00000001FF
